:020000040000FA
:06000000673002303A28CF
:08000800A000030EA100831209
:1000100081018B100B11210E8300A00E200E090010
:0C007400203084008001840A80300402E7
:10008000031C3C281230B000502183160C3085052B
:1000900087018312850187010730990000309A009B
:1000A000103083168E008312603083168F00831207
:1000B0000030831691009F008312C83083168100A0
:1000C000831231309000003083168C008312103080
:1000D0008B00831600309B001C141A088312BC008E
:1000E000851DC421831610309B001C141A0883122E
:1000F000BD00722181018E018F010B118B100B103D
:100100008C018B179220311994203221B30B902847
:10011000031085190314B90DF03039020319C321F6
:10012000EA21822864000800080031110130B7007C
:100130008B132030370783169B001C141A08831278
:10014000A4001030370783169B001C141A08831272
:10015000A3000030370783169B001C141A08831273
:10016000A2008B17321CBA2822090339A200A30966
:10017000A409A50901303702031DC3283D18C3286F
:100180003D143E14662102303702031DCC28BD18F1
:10019000CC28BD143E14692103303702031DD52835
:1001A0003D19D5283D153E146C2104303702031D3E
:1001B000DE28BD19DE28BD153E146F21B70A0530B3
:1001C00037020318080098280130B600B300B400C5
:1001D000B500B70085018701B1139220B30B0A293E
:1001E000031085190314B90DF030390203192829B9
:1001F000B41F8501B41F8701B40B0A293708B6085C
:100200000319B60003190829FF3085008700B603DB
:100210009630B400311DED283111321C14292D09FE
:100220000339AD00AE09AF098B1320303707BB008F
:100230002F08BA003B2110303707BB002E08BA0048
:100240003B2100303707BB002D08BA003B218B173C
:1002500085018701B70AB60105303702031CED2876
:10026000722108003E1C08003E101030BB003D0803
:10027000BA003B2108008B133A0883161C159A001C
:1002800083123B0883169B0055309D00AA309D00C9
:100290009C1464009C1849291C1183128B170800B8
:1002A000831620309B001C141A088312C1004108D9
:1002B0000F39C200410E0F39C3000130C2080319C3
:1002C000C2000130C3080319C30008000130BD009B
:1002D00008000230BD0008000430BD0008000830EE
:1002E000BD000800BD013D1401303D0203198729FE
:1002F00002303D020319962904303D020319A52955
:1003000008303D020319B4290130BD003E145830B5
:10031000D3000512851205148510871407110714E0
:100320008712071687110A30D40008004230D30024
:100330000512851205108510871007110710871206
:10034000071287110130D40008000530D3000512D0
:1003500085120514851487100711071087160716D4
:1003600087110A30D40008000F30D300051685121B
:1003700005108510871007150714871207128715B7
:100380000A30D40008000800B601B301B4013C1CD7
:10039000CC29BC01BC14CE29BC013C143C08B600DD
:1003A0006400D229D329D429D529D6293130B41BC8
:1003B0008500B41F8501B30BD029B40BD0290310DD
:1003C000B60CB608031DD0290030BB003C08BA00AB
:1003D0003B210800851D023085190130BD008F08C2
:1003E000031908008E018F01D0080319662AD00F67
:1003F000FB29DD23662A501C420850184308D10708
:10040000031C052AFF30D100DD2356180516D61827
:10041000851656190514D6198514561A8714D61A36
:10042000071557180714D718871657190716D7191D
:10043000871551080E020318352A58180512D818C6
:10044000851258190510D8198510581A8710D81A0E
:10045000071159180710D918871259190712D919F5
:100460008711FF305002031908008F08031D080090
:10047000922051080E02031C352A56180512D61870
:10048000851256190510D6198510561A8710D61AD6
:10049000071157180710D718871257190712D719BD
:1004A000871158180516D818851658190514D81923
:1004B0008514581A8714D81A071559180714D9180B
:1004C000871659190716D91987150800D50B080082
:1004D0004630D500D40B08000130D000D1000130E7
:1004E0005302031D7A2AD61558160F30D400023055
:1004F000D300080002305302031D852AD714591473
:100500000A30D4000330D300080003305302031D27
:100510008F2AD6140530D4000430D30008000430EC
:100520005302031DA82A56155814D81460308B1393
:1005300083169B001C141A0883128B173D19013077
:10054000D400043084000530BC184730D3000800C4
:1005500047305302031DB62A3D19D0013D1908004A
:10056000D9140130D4004830D30008004830530279
:10057000031DC22AD7140130D4000530840B473044
:10058000D300080005305302031DE42A0130D400D3
:10059000BC18D92A3D19D0013D19D1013D190800D7
:1005A0005714D9140A30D4000630BD184430D30093
:1005B00008005714D9140A30D4004930BD1844300B
:1005C000D30004308400080049305302031DEE2A92
:1005D00058150130D4004A30D30008004A30530285
:1005E000031DFA2A56150130D4000630840B493019
:1005F000D300080006305302031D052BD6145815EE
:100600000530D4000B30D30008000B305302031D1B
:10061000102B5614D8140A30D4000C30D300080024
:100620000C305302031D1B2BD71559150A30D4006B
:100630000D30D30008000D305302031D252B561634
:100640000530D4000E30D30008000E305302031DD5
:100650003E2BD616D815581670308B1383169B0078
:100660001C141A0883128B17BD190130D4000430F2
:1006700084000F30BC184B30D30008004B305302BD
:10068000031D4C2BBD19D001BD190800D91501302F
:10069000D4004C30D30008004C305302031D582BBB
:1006A000D7150130D4000F30840B4B30D300080035
:1006B0000F305302031D762B0130D400BC186D2B74
:1006C000BD19D001BD19D101BD1908005715D915A3
:1006D0000A30D4001030D30008005715D9150A305D
:1006E000D4004D30D3000430840008004D30530254
:1006F000031D802BD8160130D4004E30D3000800E3
:100700004E305302031D8C2BD6160130D40010300E
:10071000840B4D30D300080010305302031D972B7B
:100720005616D8160530D4000130D30008004230E8
:100730005302031DA32BBC18D61456160130D40047
:100740004330D300080043305302031DB12BBC18C3
:10075000D81458160130D4004230BD1C4530D300A7
:10076000080044305302031DBE2B5815D8155914E8
:1007700059150130D4004230D300080045305302EF
:10078000031DCB2B56155616571457150A30D40097
:100790005830D300080058305302031DDA2BD61509
:1007A00058161430D400043084000630BC18493088
:1007B000D30008000130D300080056180516D618DB
:1007C000851656190514D6198514561A8714D61A83
:1007D000071557180714D718871657190716D7196A
:1007E0008715D601D70158180512D818851258193F
:1007F0000510D8198510581A8710D81A07115918DA
:100800000710D918871259190712D9198711D80159
:04081000D901080002
:084000000600030004000700A4
:02400E00CC33B1
:104200000100FF00FF00FF00FF00FF00FF00FF00B4
:10421000FF00FF00FF00FF00FF00FF00FF00FF00A6
:104220000100FF00FF00FF00FF00FF00FF00FF0094
:10423000FF00FF00FF00FF00FF00FF00FF00FF0086
:104240002200FF00FF00FF00FF00FF00FF00FF0053
:10425000FF00FF00FF00FF00FF00FF00FF00050060
:10426000FF00FF00FF00FF00FF00FF00FF00FF0056
:10427000FF00FF00FF00FF00FF00FF00FF00FF0046
:10428000FF00FF00FF00FF00FF00FF00FF00FF0036
:10429000FF00FF00FF00FF00FF00FF00FF00FF0026
:1042A000FF00FF00FF00FF00FF00FF00FF00FF0016
:1042B000FF00FF00FF00FF00FF00FF00FF00FF0006
:1042C0003200FF00FF00FF00FF00FF00FF00FF00C3
:1042D000FF00FF00FF00FF00FF00FF00FF00FF00E6
:1042E0003200FF00FF00FF00FF00FF00FF00FF00A3
:1042F000FF00FF00FF00FF00FF00FF00FF000000C5
:00000001FF
